:100000000C9431000C944E000C944E000C944E0055
:100010000C9453040C944E000C944E000C944E001F
:100020000C944E000C944E000C944E000C944E0018
:100030000C944E000C944E000C944E000C944E0008
:100040000C944E000C944E000C944E000C944E00F8
:100050000C944E00D502CC02CE02D002D202D802BD
:10006000D30211241FBECFE5D8E0DEBFCDBF10E024
:10007000A0E6B0E0E6E1F1E102C005900D92AE36F7
:10008000B107D9F712E0AEE6B0E001C01D92A53A83
:10009000B107E1F70E9479070C9489080C940000DD
:1000A0000E94E7029798979A939884E40E94170316
:1000B000939A85E88A95F1F70000939880E00E9472
:1000C0001703939A85E88A95F1F70000939887E0E3
:1000D0000E941703939A85E88A95F1F70000939898
:1000E00083E00E941703939A85E88A95F1F7000050
:1000F000939880E00E941703939A85E88A95F1F718
:100100000000939884E00E941703939A85E88A95EB
:10011000F1F70000939882E50E941703939A85E80F
:100120008A95F1F70000939883E00E941703939A51
:1001300085E88A95F1F70000939881E30E94170300
:10014000939A85E88A95F1F70000939882E00E94DF
:100150001703939A85E88A95F1F7000093988EE843
:100160000E941703939A85E88A95F1F70000939807
:1001700081E00E941703939A85E88A95F1F70000C1
:10018000939883E00E941703939A85E88A95F1F784
:100190000000939884E40E941703939A85E88A9557
:1001A000F1F70000939880E00E941703939A85E886
:1001B0008A95F1F700000895CF93C82F0E94E702B7
:1001C000939881E00E941703939A9398CC2311F09F
:1001D00082E001C083E00E941703939ACF910895B3
:1001E0000E94E702939881E00E941703939A9398E4
:1001F00081E00E941703939A0895CF92DF92EF92C5
:10020000FF920E94E702939885E40E941703939A55
:1002100025E82A95F1F70000939880E00E941703E3
:10022000C82ED12CE12CF12CFE2CED2CDC2CCC2476
:1002300080E00E941703C82AFE2CED2CDC2CCC2475
:1002400080E00E941703939AA7019601282BCA0108
:10025000B901FF90EF90DF90CF90089584B780931D
:10026000540214BE8898899ABA9ABB9AD798A798CC
:10027000D6988AB38F638ABB84B38F6784BBBC9ADA
:100280008B9A8C9A8D9AC49A939A949A959ABD9ABD
:10029000BF9ABE98C59AC79A8E988F9A8A980895E1
:1002A0002FB78D5FF894A89591B5986191BD81BDE8
:1002B0002FBF0895EF92FF920F931F93CF93DF9379
:1002C000E82EFB01FF24F394C82FD0E0042F10E0A8
:1002D0004F15D8F0CE018F0D911DB8010E946F0807
:1002E000282F269526952695DF01A20FB11D2C916A
:1002F00030E0BC016770772702C0359527956A9575
:10030000E2F720FD03C0F394E3CF8E2DDF91CF9170
:100310001F910F91FF90EF90089540E46CE770E01B
:100320000C945A0144E562E971E00C945A01362FAD
:10033000FB012E2F231B241748F42191DC015D9132
:10034000CD0120952523A9F380E0089581E008954B
:100350004BE06DE971E082E991E00E9497018093A2
:100360005302089548E064E870E08CE790E00E9452
:1003700097018093520208950E94A801882341F0BA
:100380000E94B20191E0811101C090E0892F08958F
:1003900080E00895EDE9F1E0119281E0E83AF80794
:1003A000D9F70895E8EAF1E01192119282E0E03580
:1003B000F807D1F70895E4E8F0E0119280E0EC3816
:1003C000F807D9F70895ECE8F0E011921192119234
:1003D000119281E0EC38F807C1F708950E94DB0123
:1003E0000C94CA014FEF50E02FEF30E0611571051A
:1003F00009F1DB016531710510F0A4E1B0E06A1B81
:100400007B0BFC01A80FB91F8191280F311D420FF2
:10041000531FEA17FB07C1F7CF01E32FFF27DF01C7
:10042000A20FB11D9D01E52FFF27DF01A40FB11D14
:10043000AD01DCCF632F7727852F9927840F911D7E
:10044000982F8827620F711D862B972B08950F9385
:100450001F93CF93DF9360E071E08CE890E00E94FF
:10046000F20190938D0180938C0168EA70E088EA34
:1004700091E00E94F201909351028093500200E0BB
:1004800010E0CEEDD1E0BE01C8018A589F4F0E9416
:100490009F06C81BD90B080F191F2097A1F700E072
:1004A00010E0C7E0D0E0BE01C8018C5A9D4F0E9409
:1004B0009F06C81BD90B080F191F2097A1F7DF91C2
:1004C000CF911F910F91089586B1866086B93098BB
:1004D000359A80B78F7180BF379A3E983F9887B121
:1004E000866087B9369A0895883230F4E82FEE0F87
:1004F0008432C0F0EE5F16C0803550F4E8EDE80FAE
:10050000E43218F4EE0FEF5F0DC0EE0FED5F0AC09E
:10051000843538F4E0EBE80FF0E0E759FF4FE08175
:1005200001C0E0E085B3EF778078E82BE5BB089564
:10053000E82FE295EF70E43028F4F0E0EB59FF4F3C
:10054000208101C020E09BB38F70822B8F73907C41
:10055000892B8BBB08951DB880916F0280FF02C06C
:100560006D9A01C06D9880915C0280FF02C06B9A09
:1005700001C06B9880916D0280FF02C06A9A01C031
:100580006A9880916E0290E08730910570F4FC01CA
:10059000E65DFF4F0C948308699A0AC0699A03C00C
:1005A000689A06C0689A709A04C08DB183608DB94C
:1005B00070988DB180658DB9089510926E02109279
:1005C0006F0210925C0210926D020C94AB0286E0F6
:1005D00080936E0210926F0281E080935C028093A0
:1005E0006D020C94AB0284E080936E0210926F0255
:1005F00010925C0210926D020C94AB02873008F0EE
:1006000086E080936E020C94AB02811181E08093AE
:100610006F020C94AB02811181E080935C020C9418
:10062000AB02811181E080936D020C94AB026C9B54
:100630006C9A8FB9779BFECF8FB108958F929F925E
:10064000BF92CF92DF92EF92FF920F931F93CF93BF
:10065000DF931F92CDB7DEB7B82EE12CF12C262FF9
:1006600030E0A90142595F4F6A01C901805A9F4F8A
:100670004C0101E010E0EB1408F08AC0C39AF601C7
:1006800080818823D1F061110CC028B3F4018081EE
:10069000A80102C0440F551F8A95E2F7242B28BBFE
:1006A00029C022B3F4018081A80102C0440F551F64
:1006B0008A95E2F7242B22BB1DC061110EC028B31E
:1006C000F4018081A80102C0440F551F8A95E2F70A
:1006D000CA018095822388BB0DC022B3F4018081BA
:1006E000A80102C0440F551F8A95E2F7CA01809500
:1006F000822382BBC398F701E35AFD4F808169834F
:100700000E941703F701E059FD4F8083C39AF60159
:10071000808169818823F1F061110EC088B3F401F2
:100720002081A80102C0440F551F2A95E2F79A01C3
:100730002095282328BB27C082B3F4012081A8017B
:1007400002C0440F551F2A95E2F79A0120952823ED
:1007500022BB19C061110CC088B3F4012081A8012B
:1007600002C0440F551F2A95E2F7842B88BB0BC0AB
:1007700082B3F4012081A80102C0440F551F2A95BD
:10078000E2F7842B82BBC3985FEFE51AF50A73CFBB
:100790000F90DF91CF911F910F91FF90EF90DF901D
:1007A000CF90BF909F908F900895EF92FF920F93FC
:1007B0001F93CF93DF931F92CDB7DEB7182F411150
:1007C0000DC098B38091600021E030E0082E01C098
:1007D000220F0A94EAF7922798BB0EC092B3A42F77
:1007E000B0E0A05ABF4F8C9121E030E001C0220F51
:1007F0008A95EAF7922792BB062F7B018E2D801BEC
:10080000811740F4F70181917F0149830E9417030A
:100810004981F4CF41110DC028B33091600081E0CF
:1008200090E0032E01C0880F0A94EAF7282728BB1E
:100830000FC022B3E42FF0E0E05AFF4F308181E097
:1008400090E0032E01C0880F0A94EAF7282722BB04
:100850000F90DF91CF911F910F91FF90EF9008952E
:100860006C9A20E030E0281790F4C498F901E35A1C
:10087000FD4F90819FB9F901E059FD4F779903C071
:100880009FB19083FBCFC49A2F5F3F4FECCF089569
:1008900088E085BD85B5836085BD8CE783BD89B75C
:1008A000806889BF08951F920F920FB60F9211248E
:1008B0002F938F939F93AF93BF9380915902909101
:1008C0005A02873E934050F48091590290915A0207
:1008D000019690935A028093590217C010925A02BF
:1008E000109259028091550290915602A0915702A0
:1008F000B09158020196A11DB11D809355029093AD
:100900005602A0935702B0935802BF91AF919F91A6
:100910008F912F910F900FBE0F901F901895C29836
:100920002FE788E391E0215080409040E1F700C03C
:100930000000C29A8FE097E20197F1F700C0000033
:100940000895CF93DF9300D01F92CDB7DEB76983B0
:100950008A839B830E94DD0220EF20935D029B81AE
:1009600090935E028A8180935F0269816093600246
:1009700084E00F900F900F90DF91CF910C94300492
:10098000CF93DF9300D0CDB7DEB789839A830E94DF
:10099000DD022FE020935D029A8190935E028981AF
:1009A00080935F021092600284E00E943004809184
:1009B00073020F900F90DF91CF9108956AEF89E055
:1009C00090E00E94A10467EC8AE090E00E94A104FC
:1009D0006FE08BE090E00E94A1046DEA8CE090E073
:1009E0000E94A10462E28DE090E00E94A10461E017
:1009F0008EE090E00E94A1046AE08FE090E00E9407
:100A0000A10460E080E190E00E94A10460E881E13F
:100A100090E00E94A1046FE782E190E00E94A104AF
:100A20006FEF85E090E00E94A1046FEF86E090E018
:100A30000E94A1046FEF87E090E00E94A10460E0B3
:100A400088E090E00E94A1046AE081E090E00E94CA
:100A5000A10460E082E090E00E94A10460E083E0F5
:100A600090E00E94A10460E084E090E00E94A10474
:100A70006AE08AE190E00E94A1046AE08BE190E0E4
:100A80000E94A10461E080E094E00E94A10463E17F
:100A900084E094E00E94A10468E885E094E00E946C
:100AA000A10461E081E094E00E94A10483E094E06D
:100AB0000E94C0048331D1F762E081E094E00E949B
:100AC000A10483E094E00E94C0048431D1F708952A
:100AD00083E094E00E94C004873121F481E0809398
:100AE000750002C01092750080917500089583E032
:100AF00094E00C94C004CF930E947705C82F8731EF
:100B000051F0843119F41092740011C00E947705DD
:100B1000C82F873121F481E08093740008C01092BF
:100B20007400843121F00E948F040E94DE048C2F17
:100B3000CF910895CF93DF9380E294E00E94C004A8
:100B4000C82FD0E0DC2FCC2781E294E00E94C004C3
:100B50009E01280F311DC901DF91CF910895CF93D8
:100B6000DF9382E294E00E94C004C82FD0E0DC2F23
:100B7000CC2783E294E00E94C0049E01280F311D1F
:100B8000C901DF91CF910895CF93DF9384E294E080
:100B90000E94C004C82FD0E0DC2FCC2785E294E06F
:100BA0000E94C0049E01280F311DC901DF91CF9121
:100BB0000895CF9386E294E00E94C004C82F87E294
:100BC00094E00E94C0042C2F30E0322F2227A9018C
:100BD000482BCA01CF910895CF93DF9388E294E028
:100BE0000E94C004C82FD0E0DC2FCC2789E294E01B
:100BF0000E94C0049E01280F311DC901DF91CF91D1
:100C00000895CF93C82F692F84E294E00E94A10435
:100C10006C2F85E294E0CF910C94A104CF93C82F60
:100C2000692F88E294E00E94A1046C2F89E294E08D
:100C3000CF910C94A1046F927F928F929F92AF926A
:100C4000BF92CF92DF92EF92FF920F931F93CF93B9
:100C5000DF93782E0E94D905009709F460C024E044
:100C6000271510F464E0762E272D30E082179307C5
:100C700008F4782E0E94EC056C019F705C0140EA3C
:100C8000B41A072D10E09801280F391F2130304188
:100C900018F4C0E0D0E036C0C0E0D0E1C81BD90BEA
:100CA00048018C1A9D0A612CE62CF12CEC16FD06ED
:100CB00058F4C7018A0D9B1D0E94C004F701EF572D
:100CC000FD4F80836394F0CFB12C8B2D90E088157D
:100CD000990560F47C01EC0EFD1E905A0E94C00440
:100CE000F701EF57FD4F8083B394EFCFC8018C0D10
:100CF0009D1D0E940E0660E481E094E00E94A10424
:100D0000872D0EC0C71590F7C5018C0F9D1F0E943F
:100D1000C004FE01EF57FD4F80832196F3CF80E0A2
:100D2000DF91CF911F910F91FF90EF90DF90CF90C7
:100D3000BF90AF909F908F907F906F9008956F922B
:100D40007F928F929F92AF92BF92CF92DF92EF925B
:100D5000FF920F931F93CF93DF937C018B010E942F
:100D60009A05EC01009709F45AC00E94C4056C0171
:100D70009C013F70590140ECB41A0C171D0708F490
:100D8000E801C9018C0F9D1F8130904118F400E0EB
:100D900010E036C0612C70E1772E621A730A4E01A2
:100DA0008618970800E010E0F701E00FF11F60815E
:100DB000C501800F911F0E94A1040F5F1F4F0615F0
:100DC000170590F300E010E06E0C7F1C0815190564
:100DD00059F0F301E00FF11F6081C801905C0E949F
:100DE000A1040F5F1F4FF2CFC6018C0F9D1F0E9401
:100DF000010660E281E094E00E94A104CE0111C0EE
:100E00000C171D0789F3F701E00FF11F6081C50181
:100E1000800F911F0E94A1040F5F1F4FF1CF80E050
:100E200090E0DF91CF911F910F91FF90EF90DF90B5
:100E3000CF90BF90AF909F908F907F906F900895CC
:100E4000FC018081A0918002882361F0A032E0F74C
:100E500081E08A0F80938002B0E08191AB57BD4F53
:100E60008C93EFCF6A2F70E085E892E00E949F0696
:100E7000109280020895DC018C91E0918002882319
:100E800061F0E032E0F781E08E0F80938002F0E0C5
:100E90008D91EB57FD4F8083EFCFE03248F481E036
:100EA0008E0F80938002F0E0EB57FD4F8AE0808345
:100EB0006091800270E085E892E00E949F061092A7
:100EC00080020895E0918002E03248F481E08E0FC4
:100ED00080938002F0E0EB57FD4F8AE080836091C1
:100EE000800270E085E892E00E949F0610928002E6
:100EF00008951092520210925302ACE7B0E0E4E879
:100F0000F0E08FEF8D93119220E0EC38F207D1F7EB
:100F1000EDE9F1E080E09FE02FEF8A3021F0DF0182
:100F20001B972C9302C090939C0111928F5F8B3082
:100F3000A1F70E942E010E94F3020E9448040E9421
:100F400064020E948F040E94DE040E945000789484
:100F500009E110E0C1E0D0E00E947B0580915902D8
:100F600090915A02B8010E945B08892B29F4809164
:100F7000740081110E94D9050E94BC01882341F0B0
:100F80000E9427020E94DB010E94CA010E94D20136
:100F9000349B50C08091530281114CC024B185B163
:100FA000349A30E0382B3093910120939001409196
:100FB0008E0180918F01483271F5A82FB0E0AA0F01
:100FC000BB1FA855BE4F4D915C911197420F531F07
:100FD0004D935C93A82FA695A695A695B0E0A35631
:100FE000BE4F282F2770AE0102C0440F551F2A950F
:100FF000E2F79C91942B9C930E94920180938F0125
:101000000E94740210928E018FE19EE40197F1F725
:1010100000C000000FC0E82FF0E0EE0FFF1FE85502
:10102000FE4F80819181820F931F918380834F5F58
:1010300040938E01869990CF8091520281118CCF7E
:101040000E94FD00609378007093790080937A008D
:1010500090937B0020917600223049F540917700F3
:1010600024E0429FF0011124EA58FF4F668B778BF2
:10107000808F918F10927600E42FE695E695E695A5
:10108000F0E0EA58FF4F242F2770CE0102C0880FEE
:10109000991F2A95E2F79C018685822B8687842FEB
:1010A0000E948D01809377000E94980255CF2F5F98
:1010B0002093760051CFAA1BBB1B51E107C0AA1F8A
:1010C000BB1FA617B70710F0A61BB70B881F991FE9
:1010D0005A95A9F780959095BC01CD01089597FB8D
:1010E000072E16F4009407D077FD09D00E945B0804
:1010F00007FC05D03EF4909581959F4F089570951B
:1011000061957F4F0895EE0FFF1F0590F491E02D3C
:061110000994F894FFCFE2
:0E111600040304050110003020484952530024
:00000001FF
